:020000040000FA
:0400000072303A28F8
:08000800A000030EA100831209
:1000100005191028831601178312B23081002B288E
:1000200083160113831203140B190310A80DA90DD5
:10003000AA0DAB0DAC0DAC16FF302C02031D2B2806
:10004000FA302B02031D2B2831152A08AF0029088E
:10005000AE002808AD008B100B11210E8300A00EFE
:04006000200E090065
:0C007400203084008001840A6030040207
:10008000031C3C281230B000DD2183160C3085059E
:1000900087018312850187010730990000309A009B
:1000A000103083168E008312603083168F00831207
:1000B0000030831691008312C830831681008312AA
:1000C00031309000003083168C00831210308B008A
:1000D000831600309B001C141A088312BC00831680
:1000E00010309B001C141A088312BD0002228101EB
:1000F0008E018F010B118B100B108C018B178F2031
:1001000031199220BF21B30B8D28031085190314D8
:10011000B90DF03039020319682103227F286400E9
:100120003210080031110130B7008B13203037072F
:1001300083169B001C141A088312A4001030370782
:1001400083169B001C141A088312A300A600023019
:10015000A6060030370783169B001C141A0883126A
:10016000A200A7000130A7068B17321CBD28220968
:100170000339A200A309A409A50924082F02031D1D
:10018000622923082E02031D112922082D02031DB6
:10019000622901303702031DD2283D18D2283D14B0
:1001A0003E14EE2102303702031DDB28BD18DB2888
:1001B000BD143E14F12103303702031DE4283D191C
:1001C000E4283D153E14F22104303702031DED28CA
:1001D000BD19ED28BD153E14F32105303702031D6E
:1001E000F6283D1AF6283D163E14F4210630370253
:1001F000031DFF28BD1AFF28BD163E14F521073048
:100200003702031D08293D1B08293D173E14F6211E
:1002100008303702031D1129BD1B1129BD173E14DB
:10022000F72126082E02031D622927082D02031D2F
:10023000622901303702031D22293D1C22293D106D
:100240003E14F82102303702031D2B29BD1C2B2937
:10025000BD103E14FB2103303702031D34293D1D20
:1002600034293D113E14FC2104303702031D3D2981
:10027000BD1D3D29BD113E14FD2105303702031D72
:1002800046293D1E46293D123E14FE210630370206
:10029000031D4F29BD1E4F29BD123E14FF210730FB
:1002A0003702031D58293D1F58293D133E140022D3
:1002B00008303702031D6129BD1F6129BD133E149B
:1002C00001226229B70A0230370203180800952874
:1002D0000130B600B300B400B500B7008501870156
:1002E000B1138F20B30B8E29031085190314B90D98
:1002F000F03039020319B529B41F8501B41F8701F5
:10030000B40B8E293708B6080319B60003198C29D7
:10031000FF3085008700B6039630B400311D712987
:100320003111321C98292D090339AD00AE09AF09EE
:100330002F1C71298E018F010C1C71290C102E1E8F
:1003400071298B1320303707BB002F08BA00C82152
:1003500010303707BB002E08BA00C821003037071D
:10036000BB002D08BA00C8218B1785018701B70A89
:10037000B60102303702031C7129022208003E1C1C
:1003800008003E101030BB003D08BA00C82108002C
:100390008B133A0883161C159A0083123B088316A8
:1003A0009B0055309D00AA309D009C1464009C1851
:1003B000D6291C1183128B170800FF30D40002309D
:1003C000D5000C30D600BA30D7003730D800DA303C
:1003D000D9006F30DA00B830DB0008000130BD0012
:1003E00008000800080008000800080008000800CD
:1003F00085018701080008000800080008000800BF
:1004000008000800080001303D05031908005C18C9
:100410000516DC1885165C190514DC1985145C1AA0
:100420008714DC1A07155C1B0714DC1B87165D1884
:100430000716DD188715E6300E02031C292A05165B
:1004400085160514851487140715071487160716D3
:1004500087158F08031908008F018501870154084B
:10046000DE00B622D4005508DE00B622D5005608BC
:10047000DE00541CB622D6005708DE00D41CB6227B
:10048000D7005808DE00541DB622D8005908DE00F7
:10049000D41DB622D9005A08DE00541EB622DA0056
:1004A0005B08DE00D41EB622DB00CA0B5F2A5408AC
:1004B000CA00D4185C14D41E5C10D41D5C10CB0B85
:1004C000692A5508CB00D51ADC14551DDC10551FC0
:1004D000DC10CC0B732A5608CC00561A5C15561F3C
:1004E0005C11D61D5C11CD0B7D2A5708CD00571A23
:1004F000DC15D71FDC11D71DDC11CE0B872A58085D
:10050000CE00D81B5C16D81F5C12D81C5C12CF0B17
:10051000912A5908CF00591ADC16591EDC12D91F2E
:10052000DC12D00B9B2A5A08D000DA195C17DA1DAE
:100530005C135A1E5C13D10BA52A5B08D1005B1A11
:10054000DC175B1EDC13DB1FDC13D20BAD2A560855
:10055000D200D51B5D14D71F5D10D30BB52A5708E9
:10056000D300D61BDD14D81FDD100800C001DE0843
:100570000319DE035E184014DE1A40144008C0015F
:100580005E1C4014DE1E4014C005C00C5E0C08004A
:084000000F000300020006009E
:02400E00CC33B1
:10420000010078007A007C007E007B0079007F004E
:104210007D007A0078007E007C00FF00FF00FF0038
:104220000000F200F600FA00FE00F200F600FA00CC
:10423000FE00F200F600FA00FE00FF00FF00FF00A3
:10424000010005000500050005000900090009003E
:1042500009000D000D000D000D00FF00FF00FF0024
:10426000FF00FF00FF00FF00FF00FF00FF00FF0056
:10427000FF00FF00FF00FF00FF00FF00FF00FF0046
:10428000FF00FF00FF00FF00FF00FF00FF00FF0036
:10429000FF00FF00FF00FF00FF00FF00FF00FF0026
:1042A000FF00FF00FF00FF00FF00FF00FF00FF0016
:1042B000FF00FF00FF00FF00FF00FF00FF00FF0006
:1042C000FF00FF00FF00FF00FF00FF00FF00FF00F6
:1042D000FF00FF00FF00FF00FF00FF00FF00FF00E6
:1042E000FF00FF00FF00FF00FF00FF00FF00FF00D6
:1042F000FF00FF00FF00FF00FF00FF00FF00DD00E8
:00000001FF
